:100000000EC013C013C011C010C00FC00EC00DC071
:100010000CC00BC00AC009C008C007C006C011242C
:100020001FBECFEDCDBF2ED03AC0EACF1F920F92A8
:100030000FB60F9211248F939F93DF93CF930F925C
:10004000CDB7DEB78FEF8983AC98B49B02C0C49A5A
:1000500003C088E086BBC498BC9A8981982F9150D0
:1000600099838823D1F7C498BC9880E28ABFAC9A60
:100070000F90CF91DF919F918F910F900FBE0F90B6
:100080001F901895BB9AC39AAC9A80E28ABF8BB72F
:1000900080628BBF789480E385BF8895FDCFF8940C
:0200A000FFCF90
:00000001FF
